:100000000C9463000C948B000C948B000C948B006C
:100010000C948B000C948B000C9462190C9488182F
:100020000C948B000C948B000C948B000C948B0024
:100030000C948B000C948B000C948B000C948B0014
:100040000C943E180C948B000C9430190C940A19E3
:100050000C948B000C948B000C948B000C948B00F4
:100060000C948B000C948B000000000023002600F1
:10007000290000000008000201000003040700003E
:100080000000000000000200000000250028002BF6
:100090000000000000240027002A000404040404D7
:1000A0000404040202020202020303030303030125
:1000B00002040810204080010204081020010204FC
:1000C000081020006C1911241FBECFEFD8E0DEBF4E
:1000D000CDBF24E0ACEFB1E001C01D92AD31B2075D
:1000E000E1F711E0A0E0B1E0ECEFF7E302C005902A
:1000F0000D92AC3FB107D9F710E0C3E6D0E004C0E1
:100100002197FE010E94C51BC236D107C9F70E9484
:10011000BB190C94FC1B0C94000020912B02222391
:1001200061F02FB7F89430912B02313049F43DB390
:1001300030932A023DB33DBB2FBF8CBD9DBD0895BA
:1001400020932A02FACFE0911B04E350E93028F40F
:10015000F0E0EF51FE4F8081089580E00895E09136
:10016000CC039091D003992301F1803248F491E0BF
:100170009E0F9093CC03F0E0E553FD4F90E1928306
:100180002091CD033091CE03280F311D3093CE0343
:100190002093CD03E091CC0391E09E0F9093CC038C
:1001A000F0E0E553FD4F828302C0EB3898F30895E9
:1001B00092E09093CD028093CE0287FD0BC081E048
:1001C0008093D0031092CE031092CD039093CC0372
:1001D0000C94AF001092D00384E08093CC03109273
:1001E000D00281E0F5CF90E0FC01E155FF4F249172
:1001F00085569F4FFC018491882399F090E0880FE9
:10020000991FFC01EF56FF4FA591B491FC01E957EE
:10021000FF4F859194918FB7F894EC91E22BEC937A
:100220008FBF08950F931F93CF93DF93EC018C0141
:10023000060F111DC017D10721F089910E94AF0050
:10024000F9CFDF91CF911F910F910895833081F005
:1002500028F4813099F08230A9F008958730A9F010
:100260008830C9F08430B1F4809180008F7D03C064
:10027000809180008F7780938000089584B58F7778
:1002800084BD089584B58F7DFBCF8091B0008F77BA
:100290008093B00008958091B0008F7DF9CF1F93B7
:1002A000CF93DF93282F30E0F901EE58FF4F849170
:1002B000F901E155FF4FD491F901E556FF4FC49183
:1002C000CC23A9F0162F81110E942601EC2FF0E01B
:1002D000EE0FFF1FE957FF4FA591B4918FB7F89428
:1002E000EC91111108C0D095DE23DC938FBFDF9114
:1002F000CF911F910895DE2BF8CF3FB7F8948091EE
:10030000100290911102A0911202B091130226B531
:10031000A89B05C02F3F19F00196A11DB11D3FBF3D
:10032000BA2FA92F982F8827BC01CD01620F711D0C
:10033000811D911D43E0660F771F881F991F4A9505
:10034000D1F708958F929F92AF92BF92CF92DF9292
:10035000EF92FF926B017C010E947D014B015C01D9
:10036000C114D104E104F104B9F00E947D016819BF
:1003700079098A099B09683E73408105910580F3DC
:1003800021E0C21AD108E108F10888EE880E83E066
:10039000981EA11CB11CE4CFFF90EF90DF90CF908E
:1003A000BF90AF909F908F900895AF92BF92CF92E1
:1003B000DF92EF92FF920F931F93CF93DF936C0125
:1003C0007B018B01040F151FEB015E01AE18BF0806
:1003D000C017D10759F06991D601ED91FC910190B8
:1003E000F081E02DC6010995892B79F7C501DF91D0
:1003F000CF911F910F91FF90EF90DF90CF90BF9022
:10040000AF900895FC01538D448D252F30E0842F4B
:1004100090E0821B930B541710F0CF96089501972C
:100420000895FC01918D828D981761F0A28DAE0F19
:10043000BF2FB11D5D968C91928D9F5F9F73928FA0
:1004400090E008958FEF9FEF0895CF92DF92EF92A3
:10045000FF920F931F93CF93DF937C018C01060FC4
:10046000171FEC016E01CE18DF080C171D0709F4E9
:100470003DC02FB7F8948091140290911502A0917D
:100480001602B09117022FBF809334029093350269
:10049000A0933602B09337028CE292E00E941102E0
:1004A00097FF2EC02FB7F8948091140290911502F7
:1004B000A0911602B09117022FBF409134025091C3
:1004C00035026091360270913702841B950BA60BA2
:1004D000B70B40913002509131026091320270911D
:1004E000330284179507A607B707B0F2C601DF915C
:1004F000CF911F910F91FF90EF90DF90CF900895D3
:100500008993B0CFFC01918D828D981731F0828D47
:10051000E80FF11D858D90E008958FEF9FEF08950E
:10052000FC01918D228D892F90E0805C9F4F821B72
:1005300091098F73992708958CE292E00E949002AE
:1005400021E0892B09F420E0822F0895FC01A48D7D
:10055000A80FB92FB11DA35ABF4F2C91848D90E0E5
:1005600001968F739927848FA689B7892C93A089C8
:10057000B1898C91837080648C93938D848D981352
:1005800006C00288F389E02D80818F7D80830895E5
:10059000EF92FF920F931F93CF93DF93EC0181E0D3
:1005A000888F9B8D8C8D98131AC0E889F98980817A
:1005B00085FF15C09FB7F894EE89FF896083E889AD
:1005C000F98980818370806480839FBF81E090E09F
:1005D000DF91CF911F910F91FF90EF900895F62E2C
:1005E0000B8D10E00F5F1F4F0F731127E02E8C8DC6
:1005F0008E110CC00FB607FCFACFE889F98980810B
:1006000085FFF5CFCE010E94A602F1CFEB8DEC0F56
:10061000FD2FF11DE35AFF4FF0829FB7F8940B8F27
:10062000EA89FB8980818062CFCFCF938091F203EA
:1006300083508D3150F09091F3038EE1890F2FE1BB
:100640002093F2039F5F9093F3038093D403E09190
:10065000F203F0E08D3108F08CE18E5FA3EDB3E0A2
:1006600090E021E03D91930F2F5F8217D8F7EF5272
:10067000FC4F9183C0E08091F2038C1758F0EC2F6F
:10068000F0E0EF52FC4F61818CE292E00E94C802E0
:10069000CF5FF1CF83E08093F203CF910895CF93A2
:1006A000C82F8091F2038F3128F08F5F8093F2037F
:1006B0000E9415038091F203E82FF0E0EF52FC4F07
:1006C000C1838F5F8093F203CF910895CF93DF931F
:1006D000EC01888D8823B9F0AA89BB89E889F9895A
:1006E0008C9185FD03C0808186FD0DC00FB607FC8F
:1006F000F7CF8C9185FFF2CF808185FFEDCFCE01C2
:100700000E94A602E9CFDF91CF91089580912B023C
:10071000882361F09FB7F89420912B0280912A02E0
:10072000213019F48DBB9FBF08958FBF08958EBDF2
:1007300000000DB407FEFDCF8EB508951F93CF9333
:10074000DF93182F83E590E00E948D00C8EFD3E07F
:1007500060E08C850E944F01812F80680E94970382
:1007600080E00E949703182F61E08C850E944F0162
:100770000E948603812FDF91CF911F9108950F93DF
:100780001F93CF93DF93082F162F83E590E00E94ED
:100790008D00C8EFD3E060E08C850E944F01802F70
:1007A0000E949703812F0E94970361E08C850E942D
:1007B0004F01DF91CF911F910F910C948603CF933E
:1007C000DF93D82FC62F0E949E03682F6C2B8D2F8E
:1007D000DF91CF910C94BF03CF93DF93D82FC62F17
:1007E0000E949E03C0956C2F68238D2FDF91CF91BF
:1007F0000C94BF0388E20E949E03982F937093305D
:1008000029F0682F636088E20C94BF030895FF927B
:100810000F931F93CF93DF93082FF62E172F83E5A7
:1008200090E00E948D0060E0809104040E944F01DE
:1008300082E10E949703CF2DD12F0C0F1D2F111D88
:10084000C017D10721F089910E949703F9CF61E089
:10085000809104040E944F01DF91CF911F910F916D
:10086000FF900C948603EF92FF920F931F93CF9308
:10087000DF937C01C62F8A0160E082E00E94BF0303
:1008800064E08AE00E94BF0360E884E10E94DF0325
:10089000B7018C2F0E94070463E082E00E94BF032F
:1008A000C8E8D3E18AE00E949E0382FD04C021973C
:1008B000C9F783E00FC060E082E00E94BF0384E4D8
:1008C0000E949E03F801808382E40E949E03F80147
:1008D000818380E0DF91CF911F910F91FF90EF9086
:1008E00008952F923F924F925F926F927F928F92D4
:1008F0009F92AF92BF92CF92DF92EF92FF920F93AF
:100900001F93CF93DF9300D0CDB7DEB7982E562E2E
:100910003A01422E80E0C114D10411F0F601808129
:100920003A2C329420EF3222380E60E082E00E94AE
:10093000BF036FE788E00E94BF0360E884E10E9484
:10094000DF03B301842D0E940704632D8AE10E9416
:10095000BF03692D82E00E94BF03FCE09F1204C028
:1009600060E88AE10E94DF0390ED692E97E0792E1E
:1009700088E00E949E03982F952141F480FD04C0D9
:1009800081E0681A7108A1F783E0A6C08CE00E949C
:100990009E03382E837109F0B4C00115110509F4C6
:1009A00066C0E114F10409F462C084E10E949E0370
:1009B000B82EF70180818B1508F4A5C0B082BB204A
:1009C00009F44BC083E590E00E948D0060E08091C7
:1009D00004040E944F01BA9482E90E9497033801EF
:1009E000212C44244394512C2B1438F5211020C081
:1009F000AA20F1F08A2D90E0912C883048F49201E1
:100A0000082E01C0220F0A94EAF7922A0196F5CF28
:100A100082E90E949703992D9095F80120819223F5
:100A20008921892B80832394FFEF6F1A7F0ADCCF03
:100A300082E90E949703F301F5CFC8018B0D911D48
:100A40005C0180E00E949703F501808361E0809162
:100A500004040E944F010E94860388E10E949E03C5
:100A60008770B82EC114D10411F0F601808382E0A2
:100A700033FC32C00115110509F447C0E114F1043B
:100A800009F443C0882009F440C0F7016081613057
:100A900029F4F4E0BF123BC08FEF1EC06230B8F102
:100AA000B11035C06250AE014F5F5F4FC8010E9468
:100AB0003304811111C0F7019081090F111DF80154
:100AC000329720819981291322C001501109F80120
:100AD00020819A8129131BC00F900F90DF91CF9135
:100AE0001F910F91FF90EF90DF90CF90BF90AF904C
:100AF0009F908F907F906F905F904F903F902F903E
:100B0000089581E0E9CF84E0E7CF80E0E5CF87E09A
:100B1000E3CF8F92AF92CF92DF92EF92FF920F933B
:100B20001F93CF93DF93CDB7DEB72C970FB6F89412
:100B3000DEBF0FBECDBF90E699838A83E2E0F1E08D
:100B4000DE01139681918D9381E0E830F807D1F7AB
:100B50008091F90389878091FA038A878091FB034A
:100B60008B878091FC038C87812CA12CD12CC12CEC
:100B7000F12CE12C10E000E02CE0AE014F5F5F4F64
:100B800060E18EE00E9471042C960FB6F894DEBFEF
:100B90000FBECDBFDF91CF911F910F91FF90EF90CE
:100BA000DF90CF90AF908F9008956F927F928F9249
:100BB000AF92CF92DF92EF92FF920F931F93CF935A
:100BC000DF9300D0CDB7DEB78A838B013A0160E8AE
:100BD0008CE10E94EC0387E08983812CA12CCE015B
:100BE00001966C01730121E0AE014E5F5F4F60E33F
:100BF0008CE00E947104811109C0F3018081823070
:100C0000A1F481E09981911101C080E00F900F90D3
:100C1000DF91CF911F910F91FF90EF90DF90CF90D8
:100C2000AF908F907F906F90089581E0EFCF2F92DB
:100C30003F924F925F926F927F928F929F92AF926C
:100C4000BF92CF92DF92EF92FF920F931F93CF93B9
:100C5000DF93CDB7DEB72B970FB6F894DEBF0FBE8C
:100C6000CDBF60E88CE10E94EC0344244394512CF6
:100C700083E9898333243394B12C912C992D977077
:100C80009B87892D8595859585958E5F282F229543
:100C9000207F290F2A8321E0911101C020E0222E1C
:100CA000280E66246394712C6C0E7D1E680E711CD8
:100CB00099E0981B9A8727C085E98983DECF87E969
:100CC000898346E0B42ED9CF40E74A838B819C814B
:100CD00089279D8189279E8189278F83AE01485F5F
:100CE0005F4F67E0CE0101960E943304182F8111F7
:100CF000ABC01B8653E05A8729E0222ECE0107960F
:100D00003C0130E2932EAB846A2D6295607F6A0DC0
:100D10008AE10E94BF03812CFE013B966F01AE0168
:100D2000465F5F4F7A018301222D4950510960E3EC
:100D30008CE00E947104182F8230A1F58CE10E9492
:100D40009E0385FD81C08F7109F480E2282F30E079
:100D5000492D990C550B421753070CF068C0982E7B
:100D60002150310927703327E82FE595E595E59562
:100D7000EF5F91E0211101C090E0E90F41E050E008
:100D80004C0F5D1F4E0F511DFA01A20102C0440F0E
:100D9000551F2A95E2F79081942B9083803209F0B9
:100DA0006DCF92CF811150C050E295128DCF8B81C3
:100DB000883809F03EC083E093E0EB2DF0E0E75087
:100DC000FC4F980FA1E0B0E0AC0FBD1FA80FB11D04
:100DD0002C9121938F5F8913F5CFBA8483E0B812E9
:100DE0004DC08B8581114AC0AE014D5F5F4F61E000
:100DF000C3010E943304182F811126C09B81F30187
:100E0000818198133DC09C818281981339C0808173
:100E100082FF12C03394F2E03F1609F44DCF43E055
:100E2000341609F44CCF51E0351609F421CF15E002
:100E30000BC082E094E0C1CF80930304832D880F20
:100E4000380E33943092F803812F2B960FB6F89416
:100E5000DEBF0FBECDBFDF91CF911F910F91FF90ED
:100E6000EF90DF90CF90BF90AF909F908F907F904A
:100E70006F905F904F903F902F90089511E0E4CFD6
:100E800017E0E2CF8F92AF92CF92DF92EF92FF9274
:100E90000F931F93CF93DF93CDB7DEB764970FB651
:100EA000F894DEBF0FBECDBF809106048F3F61F482
:100EB000909107049F3F41F4909108049F3F21F4D3
:100EC000909109049F3FF1F190911B049923D1F176
:100ED0009BE199838A83809107048B838091080426
:100EE0008C83809109048D83AE014A5F5F4F65E07A
:100EF000CE0101960E943304811115C01C8A85E041
:100F00008B8B812CA12CCE0144966C0101977C0126
:100F10008E010F5F1F4F27E0A80160E38CE00E9465
:100F20007104882379F0833069F482E08B8BAE0101
:100F30004D5E5F4FBE016F5F7F4F82E50E94D5051A
:100F40000E94170681E080931C0464960FB6F89403
:100F5000DEBF0FBECDBFDF91CF911F910F91FF90EC
:100F6000EF90DF90CF90AF908F9008958F92AF92D7
:100F7000CF92DF92EF92FF920F931F93CF93DF9365
:100F8000FA019081923128F17A01EB0190E3988384
:100F90008983AB014E5F5F4F62E0CE010E94330454
:100FA00081110CC088248394A12CD12CC12C8E01DA
:100FB00024E0AE0160E38CE00E947104DF91CF91E8
:100FC0001F910F91FF90EF90DF90CF90AF908F9097
:100FD000089584E0F3CFEF92FF920F931F93CF9386
:100FE000FA019081923110F490E00DC08A017B01EA
:100FF000C82F843078F4A801B7018C2F0E94B6075F
:1010000091E08111F1CF892FCF911F910F91FF9026
:10101000EF90089580911C048111EDCF0E9442074A
:101020008111E9CFE1CFCF93DF93FC01208130E044
:10103000322F22278181280F311D62307105B9F1CD
:101040003296DB01B695A79561707727109779F1F5
:10105000A130B105E9F04081842F90E0982F8827D6
:101060004181480F592F511D329680E1E901220F2D
:10107000331FD7FF17C057FF02C02F5F3F4F95E0C8
:1010800029273058440F551F815081F71197DECF23
:1010900050E040E06115710541F3408150E0542F6C
:1010A0004427E3CF57FFEECF2F5F3F4FEBCFC90170
:1010B000DF91CF910895CF938091D003882319F1C8
:1010C0008091CE02813621F48091CD030E94AF0041
:1010D000E091CC0381E08E0F8093CC03F0E0E553E8
:1010E000FD4F83E08283C0E08091CC03C81770F588
:1010F000EC2FF0E0E553FD4F62818CE292E00E941C
:10110000C802CF5FF1CFC091CC036DEF6C0F60933D
:10111000CF0270E06E5F7F4F8EEC92E00E9413086A
:101120008093CB029093CC02EC2FF0E0E553FD4F7F
:101130009283E1E0EC0FF0E0E553FD4F828383E022
:101140008C0F8093CC03CE5FEC2FC8CFCF91089546
:10115000AF92BF92CF92DF92EF92FF920F931F93C5
:10116000CF935C014115510561057105B9F1E4E8C2
:10117000F3E08F012003C001219F900D1124092E5F
:10118000000CAA0BBB0B6C017D01C40ED51EE61E24
:10119000F71EC701B60120E831E541E050E00E94AA
:1011A000A31B6B017C01CA01B9016C5F7F4F8F4F9C
:1011B0009F4F27E030E040E050E00E94A31BC62F85
:1011C000CC0FC701B60120EC38EA40E050E00E94A5
:1011D000A31BC22BF501C08372836383CF911F9140
:1011E0000F91FF90EF90DF90CF90BF90AF90089558
:1011F000CF93DF93C0910702D09108022097E1F0CE
:101200008091CF03882351F086E40E94D8008FE4B8
:101210000E94AF00DF91CF910C945B0887EE0E9493
:10122000D80080E00E94AF0080E00E94AF0088817B
:101230000E94AF008981ECCFDF91CF910895CF92CA
:10124000DF92EF92FF920F931F938A019B01FC01A3
:10125000AC014C5F5F4F60E070E0CB01982F872FAF
:10126000762F6627A1916A2B4E175F07B9F799274A
:1012700068017901CC24DD24EE246C297D298E2996
:101280009F29601771078207930708F493951F91B0
:101290000F91FF90EF90DF90CF900895CF93DF9361
:1012A000E1EDF3E093E091A312A2A4EDB3E09EE19F
:1012B000ED0119929A95E9F7908191838283DF91EC
:1012C000CF91089580E70E944E0980911B040E94EF
:1012D0004F030C9415038F92AF92CF92DF92EF924F
:1012E000FF920F931F93CF93DF93CDB7DEB7649731
:1012F0000FB6F894DEBF0FBECDBF162FE62EF12C31
:10130000A701BC01CE0101960E94EC1B41E050E018
:101310004C0F5D1F4E0D5F1D612FCE0101960E9487
:101320003304811122C082E18C8B1B8A22E0210FC1
:10133000812CA12CCE0143966C0101967C018E017B
:101340000F5F1F4FA80160E38CE00E9471048111C0
:101350000CC08C898130D1F48B898430B9F481E060
:1013600099819A3009F480E0819564960FB6F894DB
:10137000DEBF0FBECDBFDF91CF911F910F91FF90C8
:10138000EF90DF90CF90AF908F90089581E0EDCFF8
:10139000FF920F931F93CF93DF9300D000D000D024
:1013A000CDB7DEB7823010F480E01CC08B01F82E80
:1013B00080911C04882311F101151105A9F382EA1B
:1013C0008983FA8284E0F801DE01139601900D9280
:1013D0008A95E1F766E0CE0101960E946B098111C2
:1013E000E3CF81E026960FB6F894DEBF0FBECDBFE7
:1013F000DF91CF911F910F91FF9008950E944207B6
:101400008111DACFD1CFEF92FF921F93CF93DF9369
:10141000CDB7DEB762970FB6F894DEBF0FBECDBF73
:10142000182F9E012F5F3F4F790180E1F901119242
:101430008A95E9F750E0C9010E94EC1B80911B04DA
:101440008350833098F5133010F480E023C0212FAF
:101450002350330BC90163E070E00E948F1B1350CF
:10146000160F812F80958370810F0E94890581114D
:10147000ECCF80EA898B1A8B62E0CE0141960E9404
:101480006B098111E2CF60E1C7010E946B098111F4
:10149000DCCF81E062960FB6F894DEBF0FBECDBF01
:1014A000DF91CF911F91FF90EF90089540E1B70138
:1014B000812F0E94C809EECF9F92AF92BF92CF9228
:1014C000DF92EF92FF920F931F93CF93DF93A82E9B
:1014D0007B018A016A01D694C794D694C794B82E2A
:1014E000CB2DCA19D0E0CC15DD0518F599249394BD
:1014F0009B0C0E94A3008B1568F480E0DF91CF91D4
:101500001F910F91FF90EF90DF90CF90BF90AF9021
:101510009F900895BE01660F771F660F771F6E0DAF
:101520007F1D44E08B2D0E94030A882331F3B92CE0
:10153000D7CFC02FC37081E009F30E94A3008B15A1
:10154000E0F20C1B1109B701600F711F4C2F8B2D9E
:10155000DF91CF911F910F91FF90EF90DF90CF908F
:10156000BF90AF909F900C94030AEF92FF920F935D
:101570001F93CF93DF93CDB7DEB728970FB6F894BC
:10158000DEBF0FBECDBF90911B049923E1F17A011C
:101590008B01BE016F5F7F4F98E0FB0111929A951E
:1015A000E9F79FEF9B839BE09C838A838091FC01FA
:1015B0008D838091FD018E838091FE018F8348E0B1
:1015C00050E084E00E945C0A81110EC082E02896FF
:1015D0000FB6F894DEBF0FBECDBFDF91CF911F9144
:1015E0000F91FF90EF9008950115110551F0E1144E
:1015F000F10439F0A701B80186E00E945C0A882353
:1016000029F380E0E4CF85E0E2CFEF92FF921F93D1
:10161000CF93DF93CDB7DEB763970FB6F894DEBFF5
:101620000FBECDBF182F7B010E94A300811748F089
:1016300082E18B8B80911B0483508330B0F5133093
:1016400010F480E026C0212F2350330BC90163E042
:1016500070E00E948F1B1350160F812F80958370AE
:10166000810F0E9489058111ECCFAE014D5E5F4F65
:10167000BE016F5F7F4F812F0E94B6078111E1CFBE
:1016800084E0FE013196D70101900D928A95E1F731
:1016900081E063960FB6F894DEBF0FBECDBFDF9139
:1016A000CF911F91FF90EF900895AE014D5E5F4F77
:1016B000BE016F5F7F4F812F0E94EB078111E0CF4A
:1016C000C0CF1F93CF93DF93CDB7DEB728970FB668
:1016D000F894DEBF0FBECDBF182FBE016B5F7F4FEA
:1016E0000E94050B8823B9F0FE0135969E01275F05
:1016F0003F4F91919923D9F019821A821B821C8243
:101700000E94A300811788F044E0BE016F5F7F4F05
:10171000812F0E94030A28960FB6F894DEBF0FBEF1
:10172000CDBFDF91CF911F91089580E0F4CFE217F4
:10173000F307F9F6F0CF8F929F92AF92BF92DF92AC
:10174000EF92FF920F931F93CF93DF93CDB7DEB746
:10175000EA970FB6F894DEBF0FBECDBF2091070207
:1017600030910802232B09F4EDC190911B049923B9
:1017700009F4E8C1182F8091CF03882309F455C0DC
:1017800081E60E94D800812F0E94AF00111133C161
:10179000109200028091080190910901A0910A0124
:1017A000B0910B018FAB98AFA9AFBAAF8BAB9CAB2D
:1017B000ADABBEAB8FA798ABA9ABBAAB8090030221
:1017C00090900402A0900502B090060220910A02B7
:1017D000B501A401CE01C7960E94A80818AE0E94C8
:1017E000A300DD24D394D80E19821A821B821C8296
:1017F00080E018E008E00D15F0F4802F8D0D99279A
:10180000991F7C01F594E7941E2DBE016F5F7F4FF9
:101810008E2D0E94050B882309F494C189818823A9
:1018200031F00E1106C00F5FE6CF81EEAACFDE2C9D
:10183000E2CF0E2DE0CF81111F5F812F123108F40E
:1018400082E126EFF22EF80E0FEF010F0F1508F4CC
:101850007BC1BE016F5F7F4F802F0E94050B8823E5
:1018600009F470C18981853F79F4B501A401CE01E5
:1018700001960E941F09AB01BC014115510561058C
:10188000710521F4102F62C10150E0CF20910A02AE
:10189000CE018F960E94A80818AAF4CF1F5F1231BC
:1018A00009F058C171C10091000220910A02CE01D5
:1018B000C3960E94A8081CAA17501093FF01011B91
:1018C000009300021BA61CA61DA61EA685E5E82EF9
:1018D000E9A69AEAF92EFAA6E0910702F091080229
:1018E00000810DA711811EA766E070E0CE018996E8
:1018F0000E9413081A8A198A21E029832A832B83DC
:101900002C832DEE2D832E832F832887E986FA865C
:101910001B861C860D871E879F87888B80910002FF
:101920008B8B8F5F8C8B8FA58D8B88A98E8B89A9D4
:101930008F8B8AA9888F8BA9898F8CA98A8F8DA973
:101940008B8F8EA98C8F8EEE8D8F8E8F8F8F88A32D
:101950009FA999A398AD9AA399AD9BA39AAD9CA377
:101960008DA38EA38FA388A768E2CE0101960E9463
:1019700012018FEF0E94AF008FEF0E94AF008FEF38
:101980000E94AF008FEF0E94AF0048E250E060E29B
:1019900070E0CE0101960E94F51B64E0CE01019635
:1019A0000E94120164E1CE0101960E94120164E1DD
:1019B000CE0101960E94120164E0CE0101960E94C0
:1019C000120164E2CE0101960E9412010E945B089E
:1019D00081E0EA960FB6F894DEBF0FBECDBFDF916F
:1019E000CF911F910F91FF90EF90DF90BF90AF903C
:1019F0009F908F9008951130E9F544E250E060E245
:101A000070E0CE0101960E94F51B60E1CE010196C7
:101A10000E94120160E1CE0101960E94120164E26F
:101A2000CE0101960E94120164E1CE0101960E944E
:101A3000120160E1CE0101960E94120168E0CE0120
:101A400001960E94120164E0CE0101960E941201EB
:101A500068E0CE0101960E9412018FEF0E94AF0054
:101A60008FEF0E94AF008FEF0E94AF008FEF0E94B8
:101A7000AF00ACCF0E94A300082F88E0ECE0F1E0BB
:101A8000DE01119601900D928A95E1F7E1E0F0E018
:101A9000EC0FFD1FE10FF11D10811A5F1295110F60
:101AA000107E8091FF01885F180FE12EF12C9FE1DD
:101AB000E90EF11C8090080190900901A0900A01A4
:101AC000B0900B011E151F0411F00CF07FCF89A6FA
:101AD0009AA6ABA6BCA6011778F0BE01615D7F4F48
:101AE000812F0E94050B882309F473CF8FA5803FB7
:101AF00011F0853F79F41AA689A50E94AF008AA546
:101B00000E94AF008BA50E94AF008CA50E94AF0081
:101B10001F5FD8CF882381F38AA740910302509199
:101B200004026091050270910602CE018F960E9418
:101B30001F09AB01BC0120910A02CE0189960E94C7
:101B4000A808DACF80E045CF112319F01850109380
:101B5000000218E0BE016F5F7F4F812F0E94050BCE
:101B6000882381F38981803F09F098CEB501A401D3
:101B7000CE0101960E941F09AB01BC014115510520
:101B80006105710509F08FCE1092FF019BCE8F92F7
:101B9000AF92CF92DF92EF92FF920F931F93CF936A
:101BA000DF9300D000D0CDB7DEB780911B0488232F
:101BB00049F08CE0E8EFF3E0ACE0B4E001900D9286
:101BC0008A95E1F780E589831A82AE014D5F5F4F08
:101BD00062E0CE0101960E943304811110C0812C75
:101BE000A12CD12CC12CF12CE12C10E000E024E040
:101BF000AE014F5F5F4F60E38CE00E94710468E0CC
:101C000080E10E94EC039FB7F8948091180288232A
:101C100019F081508093180280911802811105C03B
:101C20008CB58F7B8CBD10922B029FBF60E08091A2
:101C300019040E944F010F900F900F900F90DF91A9
:101C4000CF911F910F91FF90EF90DF90CF90AF90C9
:101C50008F9008952F923F924F925F926F927F9252
:101C60008F929F92AF92BF92CF92DF92EF92FF92AC
:101C70000F931F93CF93DF9300D000D000D0CDB748
:101C8000DEB769835E834D83452B49F49E838D8344
:101C9000893C910520F028EC30E03E832D832C0117
:101CA000712C612C9C01A0E4BFE10E94741B28EE02
:101CB00033E040E050E00E94A31B49015A0110E0CC
:101CC00000E032EB232E30E0332E89818150990BD6
:101CD0009B838A83ED81FE816F01F12CE12CA89515
:101CE00061E084E00E944F0180910101833041F561
:101CF000E6E8F0E0F491FC83F7FDC6C083E00E94C3
:101D0000F300FC81FF2309F48EC02C81223009F0FE
:101D10009EC08091B100887F82608093B1008CE783
:101D20008093B30080921E0290921F02A092200224
:101D3000B092210280917000826080937000A4C0F4
:101D40008F3F09F0A1C083E080930101E6E8F0E055
:101D5000F491FC83FF3F09F497C0F13021F150F07A
:101D6000F23009F43EC02C8127FD8EC083E00E9432
:101D7000F300CBCF14BC15BC84B5826084BD85B59F
:101D8000816085BDEEE9F0E08491E82FF0E0EE0F90
:101D9000FF1FE957FF4F85919491F1018491809342
:101DA0001D021C82ABCF10928000109281008091A6
:101DB00081008860809381008091810081608093A0
:101DC0008100EEE9F0E08491E82FF0E0EE0FFF1FD4
:101DD000E957FF4F85919491F101849180931C0202
:101DE0008DCF1092B0001092B1008091B00082604F
:101DF0008093B0008091B10081608093B100EEE9E2
:101E0000F0E08491E82FF0E0EE0FFF1FE957FF4F5D
:101E10008591949190931B0280931A02F101849111
:101E2000809319026BCF85B5887F826085BD8CE772
:101E300087BD8092260290922702A0922802B0923B
:101E4000290280916E00826080936E001DC03C81EB
:101E5000313009F051C080918100887F816080938A
:101E6000810087EE93E090938900809388008092B0
:101E7000220290922302A0922402B0922502809125
:101E80006F00826080936F00C301B2010E94A201C3
:101E9000A89560E084E00E944F0160E083E00E942A
:101EA0004F01EA81FB810E171F072CF4C701B60111
:101EB0000E94A201A8950F5F1F4FF9810F1708F428
:101EC0000ECF26960FB6F894DEBF0FBECDBFDF91C2
:101ED000CF911F910F91FF90EF90DF90CF90BF9027
:101EE000AF909F908F907F906F905F904F903F90BA
:101EF0002F90089587EE14CF3C813230D9F3311101
:101F0000C3CF87EE95CF50E040E00C942A0ECF93DC
:101F1000C82F88E70E944E098C2F0E944F038091A2
:101F20001B040E944F030E94150363E084E690E0C7
:101F3000CF910C94830F61E084EF91E00C94830FB8
:101F4000CF92DF92EF92FF920F931F93CF93DF9385
:101F500000D000D0CDB7DEB77C01162F19821A82CF
:101F60001B821C8280911B04882309F44BC00E94B1
:101F7000A300082F123098F1F7011081818181119F
:101F800001C081E0412F480F5527551F0417150642
:101F90001CF00FEF010F080F85E60E944E0983E049
:101FA0006E0155E0C50ED11C0117D8F0BE016F5F60
:101FB0007F4F812F0E94050B882331F1812F0E94D2
:101FC0004F03CE0101967C01F70181917F010E94B0
:101FD0004F03CE14DF04C1F71F5F80E0E5CF14E0AC
:101FE000DBCF882399F00E94870F0F900F900F90FE
:101FF0000F90DF91CF911F910F91FF90EF90DF90A5
:10200000CF90089585E0EFCF83E0EDCF0E941503D8
:102010000E949B0FEACF8F929F92AF92BF92CF9276
:10202000DF92EF92FF920F931F93CF93DF9300D035
:1020300000D0CDB7DEB780911B04882371F01982E0
:102040001A821B821C82BE016F5F7F4F84E00E9458
:10205000050B811116C083E001C085E00E94870F47
:102060000F900F900F900F90DF91CF911F910F91D4
:10207000FF90EF90DF90CF90BF90AF909F908F90A8
:10208000089581E60E944E0989810E944F030E94B3
:10209000A300082F8C81813009F081C08FEF0E944E
:1020A0004F0316E0812C912C5401F12CE12C0117E7
:1020B00008F4B1C0BE016F5F7F4F812F0E94050BF6
:1020C000882349F28A81298130E0522F4427E11484
:1020D000F104D9F4982F907F7A01E92A90E0B0E0DA
:1020E000A0E0DC019927882788279927AF70BB27B4
:1020F0008B809C80982489249824B12CA12C882A38
:10210000992AAA2ABB2A1F5FD2CF482B64E0569592
:1021100047956A95E1F7452BB1F3C90134E09595F0
:1021200087953A95E1F70E944F03298180E1289F26
:10213000900111248A8182958F70822B0E944F0317
:102140008A8190E0B0E0A0E0DC0199278827882709
:102150009927AF70BB272B813C8132272327322759
:10216000A90170E060E0842B952BA62BB72B6701AB
:1021700088159905AA05BB0518F480E1C80ED11C85
:102180008D2D0E944F038A818F708C290E944F03EE
:102190008B810E944F038C810E944F03B4CF8A3001
:1021A000D0F18FEF0E944F0316E0F12CE12C0117C4
:1021B00090F1BE016F5F7F4F812F0E94050B882336
:1021C00009F449CF8981811114C09A81911111C0FC
:1021D0008B8190E0B0E0A0E0BA2FA92F982F88273C
:1021E0002C81822B9C01232B11F0F82EE92E1F5FEE
:1021F000DECF0E944F038A810E944F038E2D0E94E2
:102200004F038F2D0E944F038B810E944F038C81BF
:102210000E944F03ECCF0E9415030E949B0F20CF1A
:10222000CF93C82F89E70E944E0980911B040E941A
:102230004F030E941503CC2319F0CF910C949B0FF0
:10224000CF910895CF93DF93CDB7DEB728970FB620
:10225000F894DEBF0FBECDBFFC0187E06630F0F022
:102260009E012D5F3F4F86E0D9011D928A95E9F7C7
:102270008181898380818A8382818B8383818D831D
:1022800084818E8385818F8348E050E0BE016F5F3B
:102290007F4F8CEF0E94B50A882359F00E94870F68
:1022A00028960FB6F894DEBF0FBECDBFDF91CF9159
:1022B000089581E00E941011F3CF50E040E070E0FB
:1022C00060E089EF0E94B50A81110C94870F81E0CC
:1022D0000C94101150E040E070E060E08DEF0E943F
:1022E000B50A81110C94870F81E00C9410116830AD
:1022F00018F487E00C94870F20911B04222351F0DF
:10230000BC0148E050E086E00E945C0A811104C0F4
:1023100082E0F0CF85E0EECF81E00C9410117F9247
:102320008F929F92AF92BF92CF92DF92EF92FF92E5
:102330000F931F93CF93DF93CDB7DEB76A970FB696
:10234000F894DEBF0FBECDBF8C0187E06E3008F47D
:1023500049C080911B04882309F443C089506E3022
:1023600009F056C0833008F45FC061E084E00E9449
:102370004F010E94A300E82E2DEFF22EF80ED12C73
:102380003AE0932E45E0842E52E1752EF5E0FF15DC
:1023900008F0E7C08D2D692D0E94831B61E0992311
:1023A00039F08D2D682D0E94831B911104C060E0CF
:1023B00084E00E944F01D39490911B04992349F02B
:1023C000933038F0963008F48AC09950933008F46E
:1023D00096C082E00E94870F60E084E00E944F0177
:1023E00003C085E00E94870F6A960FB6F894DEBF9F
:1023F0000FBECDBFDF91CF911F910F91FF90EF9056
:10240000DF90CF90BF90AF909F908F907F90089576
:10241000F801E684833008F0A8CF0E94A300F82ECC
:1024200084E08F0DE0FC2AC00E94A300F82E80916A
:10243000140190911501A0911601B09117018B8B99
:102440009C8BAD8BBE8B44E0BE016D5E7F4F84E004
:102450008F0D0E94C809882379F019821A821B8285
:102460008FEF8C8344E0BE016F5F7F4F82E08F0D62
:102470000E94C809811179CF82E0B4CF44E066E0C0
:1024800074E00E94C8098823B9F31A8E198E8091CE
:102490000A048F8B80910B04888F44E0BE01695E33
:1024A0007F4F85E08F0D0E94C809882329F380E8BB
:1024B000E1FE80E01B8A1C8A1D8A1E8A8B8B44E009
:1024C000BE016D5E7F4F83E08F0D0E94C809882397
:1024D00099F219821A821B821C8284E0C2CF93E097
:1024E000C92E8C2D8F0D0E94610B882309F471CFAA
:1024F000CA942FEFC212F5CFFCEFFF0E47CF7F8AB1
:10250000AE01495E5F4FBE016F5F7F4F8F2D0E940E
:10251000EB07882309F45DCF5E013DE0A30EB11CFB
:1025200083E0C82EF50184E091919923B9F01B8ACC
:102530001C8A1D8A1E8A44E0BE016D5E7F4F8F2D6E
:102540008C0D0E94C809882309F443CFCA9484E003
:10255000A81AB108EFEFCE12E5CFCECF815021F708
:10256000F5CF2E2D2550330BC90164E070E00E9499
:102570008F1BF82EFF2049F085E08F0D0E94610B24
:10258000882309F426CFFA94F5CF60E084E00E9416
:102590004F011C821B828BE08C83F8018081898330
:1025A00081818A8382818D8383818E8384818F83DD
:1025B000858188878681898787818A8780858B87BF
:1025C00081858C8782858D8783858E8784858F879B
:1025D0008585888B40E150E0BE016F5F7F4F84E0CE
:1025E0000E945C0A882309F447CF81E00E94101101
:1025F000FBCE643018F487E00C94870F462FBC01A3
:1026000050E088EF0E94B50A8111F6CF81E00C946A
:102610001011633018F487E00C94870F462FBC012B
:1026200050E08FEF0E94B50A8111F6CF81E00C9443
:102630001011663018F487E00C94870F462FBC0108
:1026400050E08EEF0E94B50A8111F6CF81E00C9424
:102650001011CF93DF9300D000D0CDB7DEB761115A
:102660000AC087E00E94870F0F900F900F900F9085
:10267000DF91CF91089519821A821B821C82FC017E
:102680008081898344E050E0BE016F5F7F4F8BEF14
:102690000E94B50A8111E6CF81E00E941011E4CFBB
:1026A000CF93DF93CDB7DEB728970FB6F894DEBF90
:1026B0000FBECDBFFC0187E06630F0F09E012D5FBC
:1026C0003F4F86E0D9011D928A95E9F78181898380
:1026D00080818A8382818B8383818D8384818E83B1
:1026E00085818F8348E050E0BE016F5F7F4F8AEFA6
:1026F0000E94B50A882359F00E94870F28960FB6CA
:10270000F894DEBF0FBECDBFDF91CF91089580E07A
:102710000E94101144EF51E063E084EF91E00E94C9
:102720002A0E64EF71E080E090E00E94A20161E077
:1027300088EE93E00E94830FE1CF0F931F93CF9316
:10274000DF93CDB7DEB763970FB6F894DEBF0FBE49
:10275000CDBF811180931A0410921B0410921C04A7
:102760001FB7F89480911802811124C0E5EAF0E0C7
:102770008491E9EBF0E09491E82FF0E0EE0FFF1F79
:10278000EF56FF4FA591B491EC91E92321F461E05C
:102790008AE00E944F018AE00E94F3008CB58061BC
:1027A0008CBD8CB580648CBD8DE00E94F3008BE005
:1027B0000E94F300809118028F5F809318021FBF60
:1027C0009091190480911804809304049093050457
:1027D0000E94F30061E0809104040E944F01809107
:1027E00005040E94F3002091050430E0F901EE5841
:1027F000FF4F8491F901E155FF4F0491F901E5562E
:10280000FF4F14911123F1F081110E942601E12F55
:10281000F0E0EE0FFF1FE859FF4FA591B491EC9146
:102820000E2381F06FE082E00E94BF0365E070E05C
:1028300080E090E00E94A20182E00E949E0384FD5D
:10284000FBCF0BC061E0809105040E944F0165E061
:1028500070E080E090E00E94A20160E884E50E94C0
:10286000BF0366E486E50E94BF0363E088E50E943B
:10287000BF0368EE8AE50E94BF0360E48AE20E941B
:10288000BF036DE382E20E94BF030E94FA0363E08C
:1028900088E20E94EC0310911A041295107F8CE4D8
:1028A0000E949E038077181749F060E78CE40E942D
:1028B000EC03612F60778CE40E94DF030E94FA032F
:1028C00065E070E080E090E00E94A20182E08B8BE6
:1028D000AE014D5E5F4FBE016F5F7F4F86E20E948B
:1028E000D5058D7F21F40E941706882391F0ECE036
:1028F000F4E08CE0DF011D928A95E9F763960FB64C
:10290000F894DEBF0FBECDBFDF91CF911F910F9125
:102910000895E0910304EF77E13448F4F0E0E056E5
:10292000FE4F80818430F9F028F48330E1F010927A
:102930001B04E4CF8530B9F08630C9F782E18B8B78
:10294000AE014D5E5F4FBE016F5F7F4F83E00E941F
:10295000B6078111ECCF8B818E3341F08D3641F07B
:10296000823129F789E080931B04C8CF8AE0FBCF2E
:102970008BE0F9CFFF920F931F93CF93DF93EC017E
:102980008B01F42E80E00E949D136F2DC801FE0183
:102990000995DF91CF911F910F91FF900C94C70D76
:1029A0000F931F93CF93DF938C010E945E1BC82F60
:1029B000C80101960E945E1BD82FC80102960E9492
:1029C0005E1BCD1749F0C81711F0D81380E0DF91D6
:1029D000CF911F910F9108958C2FF9CF8F929F92D5
:1029E000AF92BF92CF92DF92EF92FF920F931F931D
:1029F000CF93DF9300D000D0CDB7DEB780911B041A
:102A0000882379F019821A821B821C82BE016F5FB3
:102A10007F4F84E00E94050B811114C083E00E9467
:102A2000870F0F900F900F900F90DF91CF911F9114
:102A30000F91FF90EF90DF90CF90BF90AF909F905D
:102A40008F9008958B818F3F61F344E050E06CE9F3
:102A500071E0CE0101960E94DF1B892B51F044E00A
:102A600050E068E971E0CE0101960E94DF1B892BDE
:102A700011F419821A8283E60E944E0989810E940C
:102A80004F038A810E944F03BE016F5F7F4F85E035
:102A90000E94050B882311F20981CA80DB801C810A
:102AA000BE016F5F7F4F86E00E94050B882309F40B
:102AB000B5CFCE0101965C014E0195E0890E911CC7
:102AC0007501F70181917F010E944F03E814F90419
:102AD000C1F7BE016F5F7F4F87E00E94050B88231F
:102AE00009F49CCFF50181915F010E944F03AE1460
:102AF000BF04C1F70E94A300B82EDC24CD24DC243F
:102B0000F12CE12CFE2CED2CDC2CCC24C12A18E07D
:102B1000AA24A394A00EB116C8F1BE016F5F7F4F27
:102B2000812F0E94050B882309F478CF89818111B8
:102B300009C09A81911106C09B81911103C09C81AB
:102B4000992321F10E944F038A819B81982789272D
:102B50009827B0E0A0E0BA2FA92F982F88272C81C2
:102B6000822B8C159D05AE05BF0570F48A2D0E9441
:102B70004F038A810E944F038B810E944F038C81F7
:102B80000E944F031F5FC7CF802FF1CF0E94150314
:102B900048CFCF92DF92EF92FF920F931F93CF9384
:102BA000DF93CDB7DEB728970FB6F894DEBF0FBE20
:102BB000CDBF1886E2EDF3E080E2DF011D928A9539
:102BC000E9F78CE292E00E949002181619060CF0C8
:102BD0000AC28CE292E00E9482029091D103981383
:102BE00002C260E270E082ED93E00E9425028091D3
:102BF000D403482F8D3108F04CE1242F30E0F90147
:102C0000EF52FC4F648172E0740FE3EDF3E090E06B
:102C100051E0A1919A0F5F5F7517D8F76913E1C171
:102C2000E091D303E88710920001E154EB3108F002
:102C3000FFC0F0E0E25EF94E0C94C51B39164E164B
:102C40005316621667166C167B16801618178516B3
:102C5000DF16E416E916F316F81608170D171817FD
:102C6000181718171817181718171217EE175816DD
:102C70005D1665ED73E080E593E10E94BA14289635
:102C80000FB6F894DEBF0FBECDBFDF91CF911F917D
:102C90000F91FF90EF90DF90CF90089565ED73E076
:102CA00089E293E1EACF65ED73E089E093E1E5CF56
:102CB00065ED73E089E193E1E0CF65ED73E089EFC5
:102CC00092E1DBCF65ED73E08FE891E1D6CF65ED62
:102CD00073E087E791E1D1CF86E60E944E0981E05B
:102CE0000E944F038BE00E944F0380E00E944F033D
:102CF0000E941503C4CF65ED73E08AE691E1BDCF74
:102D000065ED73E08BE090E1B8CF4B7F423021F06E
:102D100087E00E94870FB3CF8091D5038250863021
:102D200028F48091D603805D893610F088E0F1CFD9
:102D3000A90165ED73E089E092E00E94EC1B89E057
:102D4000C82E82E0D82E0EEE13E0F601F1906F014E
:102D5000C8010E94D014F81671F06F2DC8010E94AE
:102D6000661B6F2DC80101960E94661B6F2DC8015E
:102D700002960E94661B0D5F1F4F0115F4E01F07AE
:102D800021F780910902883008F087E0823008F44A
:102D900082E080931A0480910B0280930604809154
:102DA0000C028093070480910D02809308048091A7
:102DB0000E028093090481E00E94101160CF65ED3E
:102DC00073E08EEE94E159CF65ED73E080EA9FE009
:102DD00054CF87E60E944E09809109020E944F035A
:102DE00080910A0283CF65ED73E082E291E145CFE5
:102DF000833008F48DCF8091D5039091D603A091B4
:102E0000D7038093FC019093FD01A093FE01D3CFE3
:102E100065ED73E08DE591E130CF65ED73E082E61D
:102E200099E02BCF63E084E690E00E94830F27CFE8
:102E300086E06FCF8CE292E00E948202182F8630EB
:102E4000F9F48CE292E00E9411021887FE01389694
:102E500081E0809300018885833709F483C008F0FE
:102E6000D7C0813609F492C0803709F487C0863014
:102E700009F4B2C065E18CE292E00E94C802FFCE84
:102E8000823009F0B8C063E070E08DEC92E00E94FF
:102E900025028091CE02823051F48091CF0280933E
:102EA000CE0261E070E08FEC92E00E942502D090AB
:102EB000CE02D7FC20C081E08093CF030FEC12E05C
:102EC000780161E070E0C8010E942502D8018D916F
:102ED0008D01803151F461E070E0C7010E9425024C
:102EE000B3E009351B0761F702C08330C9F7D88604
:102EF000EFECF2E0ADCF1092CF030091CF02073894
:102F000008F0B8CF10E07801E3E0EE0EF11CA70165
:102F100070E060E080ED92E00E94F51BB70180ED6B
:102F200092E00E942502F701E553FD4F82818093D4
:102F3000CC02F801E553FD4F86818093CB02E090EF
:102F4000CB02F090CC02B8016E5F7F4F8EEC92E026
:102F50000E941308E816F90609F08CCFD886E0ED38
:102F6000F2E076CF83E70E94D80080E00E94AF00B5
:102F70006EE088E191E00E94120105C00E94D80035
:102F80008DE40E94AF000E945B0879CE108180E042
:102F90000E949D13183099F410E0812F0E949B0B22
:102FA000882391F0111105C080910002813408F44A
:102FB00015E01F5F183089F70E94C70D60CE812F82
:102FC0000E949B0B8111F8CF0E94F80863E084E611
:102FD00090E00E94830FF0CF0E94F8080E949B0FA0
:102FE0004ECE81E096CE8CE292E00E9490021816BE
:102FF00019060CF41FCF8CE292E00E949002181682
:1030000019060CF03CCE8CE292E00E94110237CE01
:10301000813E09F4BBCFC0F4833809F02BCF108177
:10302000113808F02CCE018107FF02C000E8011B17
:1030300083E80E94D800812F0E94AF00812F90E08A
:10304000602F885E9E4F97CF803F09F497CF873FD0
:1030500009F010CF8E010F5F1F4F87E0D8011D923E
:103060008A95E9F787EF0E94D80067E0C80183CF0F
:103070000E949C0281110C94C91508951F920F9211
:103080000FB60F9211242F933F938F939F93AF937B
:10309000BF938091140290911502A0911602B091F5
:1030A000170230910F0226E0230F2D3758F50296B4
:1030B000A11DB11D20930F0280931402909315025D
:1030C000A0931602B0931702809110029091110202
:1030D000A0911202B09113020196A11DB11D80931F
:1030E000100290931102A0931202B0931302BF91A9
:1030F000AF919F918F913F912F910F900FBE0F90A5
:103100001F90189529E8230F0396A11DB11DD2CF5A
:103110001F920F920FB60F9211242F933F934F934C
:103120005F936F937F938F939F93AF93BF93EF932F
:10313000FF9380911E0290911F02A0912002B091F6
:103140002102892B8A2B8B2BD1F190911902E091CE
:103150001A02F0911B0280818927808380911E02D0
:1031600090911F02A0912002B09121021816190619
:103170001A061B069CF480911E0290911F02A091DA
:103180002002B09121020197A109B10980931E028A
:1031900090931F02A0932002B0932102FF91EF9120
:1031A000BF91AF919F918F917F916F915F914F915F
:1031B0003F912F910F900FBE0F901F901895809107
:1031C0000101E6E8F0E0E4919FEF90930101E13026
:1031D00051F030F0E23069F060E00E944F01DECF44
:1031E00010926E00F9CF90916F009D7F90936F00C9
:1031F000F3CF909170009D7F9093700091E0909339
:10320000B0009091B100987F94609093B1001092BB
:10321000B300E2CF1F920F920FB60F9211242F939B
:103220003F934F935F936F937F938F939F93AF934E
:10323000BF93EF93FF938CE292E00E94A602FF916E
:10324000EF91BF91AF919F918F917F916F915F911E
:103250004F913F912F910F900FBE0F901F90189597
:103260001F920F920FB60F9211242F938F939F935B
:10327000EF93FF93E0913C02F0913D028081E09159
:103280004202F091430282FD1BC090818091450271
:103290008F5F8F7320914602821741F0E0914502C3
:1032A000F0E0E45DFD4F958F80934502FF91EF9133
:1032B0009F918F912F910F900FBE0F901F90189597
:1032C0008081F4CF1F920F920FB60F9211240F90AE
:1032D0000FBE0F901F901895ECE2F2E0138212825D
:1032E00088EE93E0A0E0B0E084839583A683B78363
:1032F0008EEE91E09183808385EC90E095878487C2
:1033000084EC90E09787868780EC90E0918B808BAF
:1033100081EC90E0938B828B82EC90E0958B848B98
:1033200086EC90E0978B868B118E128E138E148E06
:103330008FEF9FEF9093CA028093C902E8EFF3E00A
:1033400010A211A212A213A214A2E1EDF3E01082C6
:1033500083E081A312A213A214A215A216A2809345
:10336000CC031092CE031092CD0381E08093CF0363
:103370001092D0030895CF93DF9300D000D0CDB743
:10338000DEB7789484B5826084BD84B5816084BDE5
:1033900085B5826085BD85B5816085BD80916E00F3
:1033A000816080936E001092810080918100826024
:1033B0008093810080918100816080938100809161
:1033C00080008160809380008091B1008460809350
:1033D000B1008091B00081608093B00080917A004C
:1033E000846080937A0080917A00826080937A0072
:1033F00080917A008E7F80937A0080917A00806835
:1034000080937A001092C10084E00E94F30083E070
:103410000E94F30089E00E94F3008AE00E94F3001A
:1034200060E084E00E944F0160E083E00E944F0171
:1034300060E089E00E944F0159E0E52E52E0F52E50
:103440000EEE13E0C8010E94D014F70181937F01B2
:103450000D5F1F4F0115F4E01F07A1F780910902CE
:103460008250863080F084E08093090210920A0234
:103470008FEF9FEFDC0180930B0290930C02A093DF
:103480000D02B0930E02809109029AE09093180405
:1034900099E090931904883008F087E0823008F4AE
:1034A00082E080931A0410920B0410920A04809117
:1034B0000B028093060480910C0280930704809194
:1034C0000D028093080480910E02809309048EEF10
:1034D0008093D10380E096E9A0E0B0E08093F4030C
:1034E0009093F503A093F603B093F7038AE090E07E
:1034F000A0E0B0E08093300290933102A0933202BA
:10350000B0933302E0913C02F0913D0282E080836F
:10351000E0913802F09139021082E0913A02F09184
:103520003B0289E1808310924402E0914002F091D5
:10353000410286E08083E0913E02F0913F0280816B
:1035400080618083E0913E02F0913F02808188603B
:103550008083E0913E02F0913F0280818068808309
:10356000E0913E02F0913F0280818F7D808361E097
:1035700084E00E944F0162E370E080E090E00E94EE
:10358000A20160E084E00E944F0101E012E080911E
:103590000001882309F48AC0809109020E949D13CA
:1035A00080911B04882309F479C09091F80329EFD6
:1035B00033E080E0981709F471C0F90154892F5F56
:1035C0003F4F4081541306C08F5FF4CF86EE0E94B8
:1035D000D80054C019821A821B821C82BE016F5F00
:1035E0007F4F84E00E94050B882309F457C08B812C
:1035F0008F3F09F453C08981809301028A818093AF
:103600000202BE016F5F7F4F85E00E94050B882399
:1036100009F444C0898190E0B0E0A0E0BA2FA92F5E
:10362000982F88272A81822BBA2FA92F982F882795
:103630002B81822BBA2FA92F982F88272C81822BA0
:103640000097A105B10551F11093080200930702FC
:103650008093030290930402A0930502B0930602A4
:103660008091CF03882309F4B1CF86E60E94D80069
:1036700085E50E94AF008AEA0E94AF0080E00E94C8
:10368000AF0080E00E94AF00809101020E94AF0075
:10369000809102020E94AF000E945B080E94C70D49
:1036A00062E370E080E090E00E94A2010E949C0230
:1036B000882309F46CCF0E94C91569CFF999FECF10
:1036C00092BD81BDF89A992780B50895262FF99962
:1036D000FECF1FBA92BD81BD20BD0FB6F894FA9AF5
:1036E000F99A0FBE01960895A29FB001B39FC00141
:1036F000A39F700D811D1124911DB29F700D811D1E
:103700001124911D0895991B79E004C0991F961703
:1037100008F0961B881F7A95C9F78095089597FB46
:10372000072E16F4009407D077FD09D00E94CB1B1A
:1037300007FC05D03EF4909581959F4F08957095B4
:1037400061957F4F0895A1E21A2EAA1BBB1BFD01B4
:103750000DC0AA1FBB1FEE1FFF1FA217B307E40770
:10376000F50720F0A21BB30BE40BF50B661F771FC8
:10377000881F991F1A9469F76095709580959095A8
:103780009B01AC01BD01CF010895EE0FFF1F059015
:10379000F491E02D0994AA1BBB1B51E107C0AA1F9D
:1037A000BB1FA617B70710F0A61BB70B881F991FE2
:1037B0005A95A9F780959095BC01CD010895FB011C
:1037C000DC0104C08D910190801921F441505040DA
:1037D000C8F7881B990B0895FB01DC0102C001901A
:1037E0000D9241505040D8F70895DC0101C06D930F
:0C37F00041505040E0F70895F894FFCFDE
:1037FC0001FFFFFFFFFFFFFFEEEEEEEE0001040501
:10380C0006070203FFFFFFFF00000001F73632330B
:10381C000A0119919780200D4B084EFA280A0119BC
:10382C00006DDD0000001804FF03800000000000A4
:10383C00000000004D70FFFFFF00C3FF0000000AF6
:10384C0000000000FF00EFFF0024FEC0FFFF1999ED
:10385C00051E7FF8850C0101A6E06FFFFFFFFFFF3F
:10386C00FFFFFFFFFFFFFFFF303030357D203800BA
:10387C0000000000FFFFFFFF3005013505100801B7
:10388C00000000001C2000780300FE000103A00CC7
:10389C0006080000FF000000040300000000000008
:1038AC0007070000000000000500000000000000F9
:1038BC0001000000000000000000000000000000FB
:1038CC0000000000000000000000000000000000EC
:1038DC00021132622700002781E100000000C802BB
:0C38EC00D5010202660390021102820264
:00000001FF
